:100000000C940E050C9456050C9456050C9456054C
:100010000C9456050C9456050C9456050C945605F4
:100020000C9456050C9456050C94B10F0C9456057F
:100030000C94111E0C9456050C9456050C94560500
:100040000C9456050C9456050C9456050C945605C4
:100050000C9456050C946A1E0C9456050C94560587
:100060000C9456050C94ED070C9456050C9456050B
:100070000C9456050C9456050C9456050C94560594
:100080000C9456050C9456050C9456050C94560584
:100090000C9456050C9456050C9456050C94560574
:1000A0000C9456050C9456050C945605FF0D260E1F
:1000B0001E0F260E1E0F720E950E1E0FEC0EFB0E5F
:1000C000531453148B148B1406153A15311731172A
:1000D00051153117E214E214EB16311700171E17F1
:1000E000291E1F20212223242526272D2E742A2B6A
:1000F000141A0815171C180C12132F302804160791
:10010000090A0B0D0E0F3334311D1B061905111092
:10011000363738752C764E4B494C52504F514A4D1C
:1001200056545F6061555C5D5E57595A5B67626605
:100130006377444568696A807071727380806580F6
:1001400048463A3B3C3D3E3F4041424380808080B0
:100150007939007A7880807B7F7E8080807D808086
:10016000706339385F6C65643A20253032580A0074
:100170007573625F6C65643A20253032580A0073EB
:10018000656E6420253032583A20253032580A00F6
:1001900073656E642039443A20253032580A007263
:1001A00025303258200073656E642037303A2025A0
:1001B0003032580A0073656E642039433A20253086
:1001C00032580A00722530345820007325303258D6
:1001D00020006F6C6420747970650A006E6577206A
:1001E000747970650A000A4C6F6F702073746172C5
:1001F000742E0A000A55534220636F6E6669677554
:100200007265642E0A000A544D4B3A3863306532E9
:10021000342F4C5546413A6436613764660A0030E3
:1002200003500043003900380020006B006500795E
:100230000062006F00610072006400200063006FC4
:10024000006E0076006500720074006500720000A8
:10025000000E0374002E006D002E006B002E0000B7
:10026000000403090409025B00030100A032090431
:1002700000000103010100092111010001224000D9
:100280000705810308000A090401000103010200B7
:10029000092111010001227F0007058203080001E6
:1002A00009040200020300000009211101000122DB
:1002B0002200070583032000010705030320000136
:1002C0001201100100000008EDFE01980101010279
:1002D00000010631FF0974A1010975150026FF0010
:1002E0009520750881020976150026FF0095207576
:1002F000089102C005010902A1010901A1008501BF
:1003000005091901290815002501950875018102C3
:100310000501093009311581257F9502750881068F
:1003200009381581257F950175088106050C0A3865
:10033000021581257F950175088106C0C005010958
:1003400080A10185021601002637001A81002AB714
:1003500000751095018100C0050C0901A1018503FC
:10036000160100269C021A01002A9C0275109501B4
:100370008100C005010906A101050719E029E7155B
:100380000025019508750181029501750881010517
:1003900008190129059505750191029501750391CB
:1003A000010507190029FF150026FF0095067508AD
:1003B0008100C0636F6E73756D65723A20253034AD
:1003C000580A0073797374656D3A20253034580AE1
:1003D000000A002530325820006B6579626F617227
:1003E000643A20004C45443A20253032580A002512
:1003F000583A2530386225730A000A2020303132FD
:1004000033343536370A00290A002575002F0025B8
:1004100075005D280025640020002564002000256B
:10042000640020002564007C0025303258006D6F88
:100430007573656B6579205B62746E7C78207920BA
:100440007620685D287265702F61636C293A205BA5
:10045000006D6B5F776865656C5F74696D655F746F
:100460006F5F6D6178203D2025640A006D6B5F77BA
:100470006865656C5F6D61785F7370656564203D6C
:100480002025640A006D6B5F74696D655F746F5F32
:100490006D6178203D2025640A006D6B5F6D617889
:1004A0005F7370656564203D2025640A006D6B5F95
:1004B000696E74657276616C203D2025640A006D5A
:1004C0006B5F64656C6179203D2025640A006D6B6B
:1004D0005F776865656C5F74696D655F746F5F6D8C
:1004E0006178203D2025640A006D6B5F7768656543
:1004F0006C5F6D61785F7370656564203D20256475
:100500000A006D6B5F74696D655F746F5F6D617814
:10051000203D2025640A006D6B5F6D61785F73700C
:10052000656564203D2025640A006D6B5F696E740B
:10053000657276616C203D2025640A006D6B5F64F6
:10054000656C6179203D2025640A000A002575004C
:10055000363A20776865656C5F74696D655F746FA6
:100560005F6D61783A20000A00257500353A2077E2
:100570006865656C5F6D61785F73706565643A206E
:10058000000A00257500343A2074696D655F746F48
:100590005F6D61783A20000A00257500333A206DBE
:1005A00061785F73706565643A20000A0025750004
:1005B000323A20696E74657276616C286D73293ADF
:1005C00020000A00257500313A2064656C617928A5
:1005D0002A31306D73293A20000A092D2056616CAA
:1005E000756573202D0A004D3E004D25643E2000A8
:1005F0003F007365742064656661756C740A00431E
:100600003E200077686572652064656C74613A20ED
:10061000637572736F723D25642C20776865656C15
:100620003D25640A53656520687474703A2F2F6500
:100630006E2E77696B6970656469612E6F72672FC2
:1006400077696B692F4D6F7573655F6B6579730A99
:10065000000A092D204D6F7573656B6579202D0A91
:100660004553432F713A09717569740A313A096427
:10067000656C6179282A31306D73290A323A09692B
:100680006E74657276616C286D73290A333A096D50
:1006900061785F73706565640A343A0974696D65E1
:1006A0005F746F5F6D61780A353A09776865656CCC
:1006B0005F6D61785F73706565640A363A097768C3
:1006C00065656C5F74696D655F746F5F6D61780AF5
:1006D0000A703A097072696E742076616C75657380
:1006E0000A643A097365742064656661756C747395
:1006F0000A75703A092B310A646F776E3A092D3109
:100700000A706775703A092B31300A7067646F7729
:100710006E3A092D31300A0A7370656564203D20F8
:1007200064656C7461202A206D61785F7370656503
:1007300064202A2028726570656174202F207469F6
:100740006D655F746F5F6D6178290A003F004D3EF3
:100750002000433E20004C25640A000A092D204356
:100760006F6E736F6C65202D0A4553432F713A09E4
:10077000717569740A6D3A096D6F7573656B65798A
:100780000A000A092D204D61676963202D0A643A29
:100790000964656275670A783A096465627567205D
:1007A0006D61747269780A6B3A09646562756720D5
:1007B0006B6579626F6172640A6D3A09646562758E
:1007C00067206D6F7573650A763A0976657273698D
:1007D0006F6E0A733A097374617475730A633A0928
:1007E000636F6E736F6C65206D6F64650A302D34B6
:1007F0003A096C61796572302D34284631302D46C6
:1008000034290A506175733A09626F6F746C6F61B5
:100810006465720A003F0074696D65725F7265619C
:1008200064333228293A202530346C580A006B652D
:1008300079626F6172645F69646C653A2025580A59
:10084000006B6579626F6172645F70726F746F6361
:100850006F6C3A2025580A00686F73745F6B657976
:10086000626F6172645F6C65647328293A20255851
:100870000A000A092D20537461747573202D0A0033
:100880004743433A20352E342E30204156522D4CCA
:100890004942433A20322E302E30204156525F4199
:1008A0005243483A20617672350A004F5054494FFE
:1008B0004E533A204C554641204D4F5553454B45DC
:1008C000592045585452414B455920434F4E534FA0
:1008D0004C4520434F4D4D414E44204B45594D41D1
:1008E000505F53454354494F4E20343039360A0047
:1008F0004255494C443A203863306532342028311F
:10090000313A34333A313320536570203137203255
:10091000303231290A005649443A2030784645455C
:100920004428742E6D2E6B2E29205049443A2030D5
:1009300078393830312850433938206B6579626F07
:1009400061726420636F6E766572746572292056D9
:1009500045523A203078303130310A004445534313
:100960003A20636F6E766572747320504339382075
:100970006B6579626F6172642070726F746F636F00
:100980006C20696E746F205553420A000A092D20AD
:1009900056657273696F6E202D0A000A6D6F75734C
:1009A000653A206F66660A000A6D6F7573653A20B6
:1009B0006F6E0A000A6B6579626F6172643A206F2C
:1009C00066660A000A6B6579626F6172643A206F2D
:1009D0006E0A000A6D61747269783A206F66660A61
:1009E000000A6D61747269783A206F6E0A000A64B9
:1009F000656275673A206F6E0A000A646562756702
:100A00003A206F66660A000A0A626F6F746C6F6143
:100A10006465722E2E2E2000433E200011241FBE3E
:100A2000CFEFDAE0DEBFCDBF04B603FE28C0809171
:100A3000570490915804A0915904B0915A048730FA
:100A4000904BA740B04BD9F4109257041092580421
:100A50001092590410925A0414BE0FB6F894A89537
:100A600080916000886180936000109260000FBEEA
:100A70001092010810920008E0E0F8E3099511E0F7
:100A8000A0E0B1E0E8EBFDE402C005900D92A433D4
:100A9000B107D9F724E0A4E3B1E001C01D92A73566
:100AA000B207E1F70E94120B0C94DA260C940000B6
:100AB000FF93EF93E0913401F0913501309709F005
:100AC0000995EF91FF910895FC018591803011F017
:100AD000EFDFFBCF0895FF27E0E230E247FF0CC0D5
:100AE000419597FF09C0EDE26095709580959095CE
:100AF000611D711D811D911D27FF02C0219530E3ED
:100B000050E2AA27660F771F881F991FAA1FA417F4
:100B100010F0A41B63955A95A9F7AA3008F0A95FB5
:100B2000A05DAF93F395611571058105910541F7BE
:100B3000ED3211F4EF93F395F21718F43F93F39518
:100B4000FBCF8F91B5DFFA95E1F70895E991F9911F
:100B50008591803021F0853219F0AADFF9CF089510
:100B600020E0E89455915532C1F3503311F4689464
:100B700055915A3348F4505390F3220F022E220F0E
:100B8000220F200D250FF4CF0EF421958991999114
:100B9000533619F3533729F1533559F1BC018827DE
:100BA0009927E8945C3621F489919991689455913C
:100BB000543639F446EF7EF077FF0DC08FEF9FEF8C
:100BC0000AC055374AE039F0583540E121F0523635
:100BD00042E009F00895FF93EF937DDFEF91FF91DD
:100BE000B7CFFF93EF93FC0181918030B9F360DFC1
:100BF000FBCFFF93EF9368DFF1CFDF93CF93CDB7B8
:100C0000DEB72596A3DFCF91DF910895CF93C82F4C
:100C10001F928F938BEC91E09F938F930E94FD0521
:100C20005C9A8FE99FE00197F1F700C000008C2FDC
:100C30000E94E6078FE99FE00197F1F700C00000EE
:100C40005C980F900F900F900F90CF9108951F9385
:100C5000CF93DF931FEF0E94D207EC011150CF3FDB
:100C60009FEFD90741F48FE99FE00197F1F700C0AA
:100C700000001111F0CF5C9A85ED8A95F1F7000024
:100C80005C98DF93CF9384EC91E09F938F930E94C5
:100C9000FD050F900F900F900F90CE01DF91CF9137
:100CA0001F910895EF92FF920F931F93CF93DF93BD
:100CB000539A549A519A5B9A5C9A599A0E94BC072B
:100CC0005C9A5B9820E52A95F1F75B9A8FEF90E7A5
:100CD00022E0815090402040E1F700C000008FE901
:100CE0000E9406060E9427068A3F910569F40E9429
:100CF0002706803A910541F40E9427068038910525
:100D000019F48CED91E002C082ED91E09F938F93F6
:100D10000E94FD050F900F9005EB11E086EAE82E8A
:100D200081E0F82E8CE90E9406060E942706EC015D
:100D3000CF3F8FEFD80729F4E7E3F1E087E491E0B4
:100D40002DC08091390480FF0AC0DF93CF931F9399
:100D50000F930E94FD050F900F900F900F90CA3FC8
:100D6000D10551F780E70E9406060E942706EC0194
:100D7000CF3F8FEFD807B1F28091390480FF0AC0CE
:100D8000DF93CF93FF92EF920E94FD050F900F909B
:100D90000F900F90CA3FD10529F6CECF11928E1732
:100DA0009F07E1F75C98DF91CF911F910F91FF9022
:100DB000EF900895EF92FF920F931F93CF93DF93DD
:100DC0000E94D207F82E082F192F0F3F8FEF180718
:100DD00009F04EC080913601882309F48FC000E9E4
:100DE00011E09FE7E92E91E0F92E8DE90E940606B9
:100DF0000E942706EC01CF3F8FEFD80721F4109215
:100E0000360180E07BC08091390480FF0AC0DF9307
:100E1000CF931F930F930E94FD050F900F900F909B
:100E20000F90CA3FD10559F7809136010E940606FE
:100E30000E942706EC01CF3F8FEFD807B1F28091D7
:100E4000390480FF10C0DF93CF93809136011F9249
:100E50008F93FF92EF920E94FD050F900F900F90DD
:100E60000F900F900F90CA3FD10509F0BECFC7CFAA
:100E70009F93FF928FE991E09F938F930E94FD05CE
:100E80000F900F900F900F90E80183E0D695C795D3
:100E90008A95E1F76F2D67708C2F8F70F7FE14C065
:100EA0000E940612882319F1CF70DD27C95CDE4F3E
:100EB0000770112781E090E001C0880F0A95EAF7DA
:100EC00080959881892312C00E94061281110FC05B
:100ED000CF70DD27C95CDE4F0770112781E090E0FD
:100EE00001C0880F0A95EAF79881892B88835C9A5C
:100EF00085ED8A95F1F700005C988F2DDF91CF91F9
:100F00001F910F91FF90EF900895E82FF0E0E95CBA
:100F1000FE4F8081089580FD02C090E701C091E7F7
:100F20009093360181FF05C09091360194609093B3
:100F300036019091390490FF0CC01F928F9380E787
:100F400091E09F938F930E94FD050F900F900F905B
:100F50000F908091390480FF0EC0809136011F925E
:100F60008F9380E691E09F938F930E94FD050F90F1
:100F70000F900F900F90089583E38093CC00109210
:100F8000CD00E9ECF0E08081806980838081886019
:100F90008083EAECF0E080818063808352985A9AE3
:100FA000789408952091470180914801821759F063
:100FB00030E0F901E75BFE4F80812F5F3F4F2093C8
:100FC000470190E008958FEF9FEF08959091C8003A
:100FD00095FFFCCF8093CE0008951F920F920FB61D
:100FE0000F9211242F933F934F938F939F93EF93DF
:100FF000FF938091480190E09C012F5F3F4F40910B
:101000004701421741F03091CE00FC01E75BFE4FF3
:10101000308320934801FF91EF919F918F914F91E1
:101020003F912F910F900FBE0F901F9018958091B8
:1010300055030895CF93DF9300D01F92CDB7DEB74D
:1010400020914E04243021F523E029839B838A8359
:1010500082E08093E9008FEF9091E800815095FD48
:1010600006C095ED9A95F1F700008111F5CF8091BA
:10107000E80085FF0DC040E050E063E070E0CE0185
:1010800001960E94CA0C8091E8008E778093E80058
:101090000F900F900F90DF91CF910895CF93DF9332
:1010A00000D01F92CDB7DEB720914E04243061F5F9
:1010B00019821A821B8222E029838138910520F04F
:1010C000805891099B838A8382E08093E9008FEFA7
:1010D0009091E800815095FD06C095ED9A95F1F745
:1010E00000008111F5CF8091E80085FF0DC040E040
:1010F00050E063E070E0CE0101960E94CA0C80913E
:10110000E8008E778093E8000F900F900F90DF91AA
:10111000CF91089520914E04243051F522E0209380
:10112000E9002FEF3091E800215035FD06C035ED84
:101130003A95F1F700002111F5CF2091E80025FF45
:1011400017C020911001222341F021E02093F100EB
:1011500040E050E065E070E004C040E050E063E053
:1011600070E00E94CA0C8091E8008E778093E800BE
:101170000895CF93DF9320914E04243049F521E068
:101180002093E90021E8215059F03091E80035FD25
:1011900007C0EFE3F1E03197F1F700C00000F3CFB3
:1011A0002091E80025FF14C0EC0140E050E068E029
:1011B00070E00E94CA0C8091E8008E778093E8006E
:1011C00088E0FE01ADE4B3E001900D928A95E1F76D
:1011D000DF91CF910895CF93C0914B02C1110BC005
:1011E0000E944F1E643C79408105910520F081E00A
:1011F00080934B02C1E08C2FCF910895FF920F9303
:101200001F93CF93DF93D82F0FB607FE83C0809133
:101210004E04843081F08091030190E0019620918A
:10122000050130E0822393232091040130E08217EE
:10123000930709F0CDC00E94EB08811110C0809186
:10124000030190E001962091050130E08223932371
:101250002091040130E08217930709F0B9C00E9481
:10126000431E8C01C091E900CF709091EC00892F52
:10127000817090FD80E8C82B83E08093E90085E0D1
:10128000F82E8091EB0085FD42C08091EB0080FF3D
:101290003EC08091EE0087FF3AC08091040190919A
:1012A0000301981709F457C09091E80095FF8EC08C
:1012B000E0910101F0910201E80FF11D20818F5FA3
:1012C000909105018923809304012093F10080917E
:1012D000E80085FDE2CF8091E80080FFDECF8091BD
:1012E000E8008E778093E800F0920001D6CF8091DD
:1012F000030190E001962091050130E082239323C1
:101300002091040130E08217930709F44CC0CF709C
:10131000C093E90040910301842F90E00196209151
:10132000050130E0822393232091040130E08217ED
:10133000930709F450C0E0910101F0910201E40F1C
:10134000F11DD083809103018F5F90910501892366
:101350008093030140C08091E80085FF37C0D0939F
:10136000F10021E03091F3008091F20090E0932BA6
:10137000892B91F08091E80080FF0EC08091E800F9
:1013800085FF03C01092F100F9CF8091E8008E77BD
:101390008093E800F0920001222309F4A8CFCF70D7
:1013A000C093E90018C080910001882309F4AFCFF1
:1013B0000E94431E9C018017910711F4890161CF9F
:1013C00090910001915090930001F8CF20E0CACF96
:1013D00040910301B0CF80E0DF91CF911F910F9139
:1013E000FF90089580914D04811104C00E94360F32
:1013F0000C94930F089510924D040895089542E0BF
:1014000061EC81E00E94430C42E061EC82E00E94CA
:10141000430C42E261EC83E00C94430C8091500455
:10142000833009F453C030F4813071F0823009F414
:10143000BAC008958A3009F4A6C08B3009F478C088
:10144000893009F0C8C020C080914F04813A09F06A
:10145000C2C08091E800877F8093E80080915304A8
:1014600090915404892B21F468E08DE493E003C04B
:1014700060E080E090E070E00E94170D8091E8004D
:101480008B778093E800089580914F04813209F0B2
:10149000A2C08091530490915404892B09F09BC001
:1014A0008091E800877F8093E8008091E80082FDCA
:1014B00005C080914E048111F8CF8DC08091F1005C
:1014C000809355038091E8008B7781C080914F0411
:1014D000813A09F080C08091530490915404892B83
:1014E000A1F48091E800877F8093E8008091E80074
:1014F00080FFFCCF809111018093F1008091E80082
:101500008E778093E8000E94780C8091530490912C
:101510005404019709F05FC08091E800877F8093B1
:10152000E8008091E80080FFFCCF809110014AC064
:1015300080914F04813209F04EC080915304909104
:101540005404892B69F48091E800877F8093E80038
:101550000E94780C80915104809311010E94031421
:1015600080915304909154040197A9F58091E8006B
:10157000877F8093E8000E94780C809151048093CB
:1015800010010C94031480914F04813221F5809155
:10159000E800877F8093E8000E94780C80915204D5
:1015A00080935603089580914F04813AA1F480916D
:1015B000E800877F8093E8008091E80080FFFCCFFF
:1015C000809156038093F1008091E8008E7780939C
:1015D000E8000C94780C08958091550380934C0298
:1015E000109255030E9404120C9403140C94EC0AFC
:1015F0000E94D01D80914C04882329F00E94F91D7F
:1016000081110C942D0C08950E940D1E80914C02A6
:101610008093550308950C94040B08950C940D0BBE
:101620000C940D0BCF9384B7877F84BF0FB6F894CB
:10163000A89580916000886180936000109260009E
:101640000FBE90E080E80FB6F8948093610090930D
:1016500061000FBE8EEF98E00E94A21D86E091E02F
:101660000E949A1086E092E00E9464050E94100B8E
:101670000E9459110E94360F0E94930F78940E9485
:101680005B1180914E04843029F00E947F100E94EB
:101690000D0BF7CF84EF91E00E9464050E940E0BC2
:1016A00086EE91E00E946405C3E080914E0485308F
:1016B00019F40E94F80AF9CF0E94B91D0E945F1127
:1016C0002091E4003091E5008091490290914A0216
:1016D0002817390709F468C08091E4009091E5006B
:1016E00090934A02809349020E94EB08882309F4F0
:1016F0005BC080914E04843009F056C08091E900AF
:101700008F702091EC00922F917020FD90E8892B32
:10171000C093E9009091EB0090FF43C09091EE00E0
:1017200097FF3FC09091040120910301291709F10F
:101730002091E80025FF1DC0E0910101F091020118
:10174000E90FF11D30819F5F209105019223909355
:1017500004013093F1009091E80095FDE3CF909162
:10176000E80090FFDFCF9091E8009E779093E8002B
:10177000D9CF9091F3002091F20030E0392B232B48
:1017800081F09091E80090FF0CC09091E80095FFE7
:1017900003C01092F100F9CF9091E8009E779093EA
:1017A000E8008F708093E9000E947F107ECF292F80
:1017B000332723303105C9F060F42130310581F041
:1017C0002230310509F041C08BE590E025E632E09A
:1017D00040C021323105E1F02232310531F135C00E
:1017E00082E190E020EC32E034C09927813091050D
:1017F00049F028F0029749F5EFE1F2E005C0E1E693
:10180000F2E002C0E1E5F2E0849190E09F0121C0A6
:1018100063307105D0F4660F771FFB01ED5DFE4F5D
:101820002081318189E090E014C06330710568F453
:10183000FB01EE0FFF1FE35EFE4F20813181FB01B4
:10184000E65EFE4F808190E004C080E090E020E002
:1018500030E0FA0131832083089580E189BD82E17F
:1018600089BD09B400FEFDCF8091D8008F7D8093A3
:10187000D8008091E00082608093E0008091E000D9
:1018800081FDFCCF0895982F973068F59093E9007B
:10189000981739F07091EC002091ED005091F00014
:1018A00003C0242F762F50E021FD02C09F5FECCFB4
:1018B0003091EB003E7F3093EB003091ED003D7FA7
:1018C0003093ED003091EB0031603093EB0070937A
:1018D000EC002093ED005093F0002091EE0027FDE6
:1018E000E5CF80E008958F708093E90081E008954E
:1018F00080914F0487FF11C08091E80082FD05C0F0
:1019000080914E048111F8CF11C08091E8008B774F
:101910000BC080914E04882349F08091E80080FF3D
:10192000F8CF8091E8008E778093E80008952091A9
:10193000E4003091E50095E64091EC00842F817041
:1019400040FF23C08091E80080FD1DC080914E04BF
:10195000882399F0853099F08091EB0085FD11C0C6
:101960004091E4005091E5002417350729F3915088
:1019700011F09A01E1CF84E0089582E0089583E0B8
:10198000089581E0089580E008954091E80042FFC5
:10199000DDCF0895CF92DF92EF92FF920F931F93C6
:1019A000CF93DF93EC018B017A010E94970C811198
:1019B00035C0E114F10439F0F70180819181081BF1
:1019C000190BC80FD91FC12CD12C0115110529F1F4
:1019D0008091E80085FD18C08091E8008E778093A3
:1019E000E8000E947F10E114F10449F0F7018081C2
:1019F0009181C80ED91ED182C08285E00FC00E949D
:101A0000970C882311F30AC089918093F10001504B
:101A10001109FFEFCF1ADF0AD8CF80E0DF91CF9115
:101A20001F910F91FF90EF90DF90CF90089520913C
:101A30005504309156042617370748F06115710593
:101A400039F42091E8002E772093E80001C0B90115
:101A5000FC0120E06115710579F180914E04882325
:101A6000F1F18530F1F18091E80083FD3CC0809177
:101A7000E80082FD2EC08091E80080FFEBCF20912E
:101A8000F3008091F20090E0922B6115710551F006
:101A90008830910538F421912093F100615071094B
:101AA0000196F3CF21E0089709F020E08091E8004B
:101AB0008E778093E800CECF2111CFCF0AC08091DE
:101AC0004E04882361F0853061F08091E80083FD49
:101AD0000AC08091E80082FFF2CF80E0089582E0A2
:101AE000089583E0089581E0089520915504309190
:101AF00056042617370748F06115710539F420910F
:101B0000E8002E772093E80001C0B901FC0120E035
:101B10006115710591F180914E04882309F440C04C
:101B2000853009F43FC08091E80083FD3DC080917D
:101B3000E80082FD2FC08091E80080FFE9CF20916E
:101B4000F3008091F20090E0922B6115710559F03D
:101B50008830910540F424912093F1003196615032
:101B600071090196F2CF21E0089709F020E08091F9
:101B7000E8008E778093E800CBCF2111CCCF0AC04C
:101B800080914E04882361F0853061F08091E800F7
:101B900083FD0AC08091E80082FFF2CF80E00895C3
:101BA00082E0089583E0089581E008951F93CF9324
:101BB000DF93CDB7DEB7AA970FB6F894DEBF0FBE9E
:101BC000CDBFEFE4F4E08091F100819324E0E735AC
:101BD000F207C9F70E940E0A8091E80083FF2EC128
:101BE00080914F0490915004492F50E04A305105A4
:101BF00008F024C1FA01EA5AFF4F0C94C02680383D
:101C000021F0823809F01AC108C080914B049091EC
:101C10004C04992389F082600FC0809153048F7027
:101C2000873008F00BC18093E9008091EB0085FBC1
:101C3000882780F91092E9009091E800977F9093AF
:101C4000E8008093F1001092F100D1C0282F2D7F81
:101C500009F0F4C0882319F0823061F0EFC0809160
:101C60005104813009F0EAC0933009F080E080939C
:101C70004C042EC08091510481112AC080915304DC
:101C80008F702FEF280F263008F0D8C08093E9001E
:101C90002091EB0020FF1CC0933021F48091EB00D9
:101CA000806214C09091EB0090619093EB0021E072
:101CB00030E0A90102C0440F551F8A95E2F7409316
:101CC000EA001092EA008091EB0088608093EB00BC
:101CD0001092E9008091E800877F8093E8000E94DD
:101CE000780CACC08111AAC0109151041F7780916B
:101CF000E3008078812B8093E3008091E800877F68
:101D00008093E8000E94780C8091E80080FFFCCF6F
:101D10008091E30080688093E300111102C082E0AB
:101D200001C083E080934E0489C08058823008F05F
:101D300085C080915104909152048C3D53E09507E9
:101D400079F583E08A838AE289834FB7F894DE01CC
:101D5000139620E03EE051E2E32FF0E0509357006D
:101D6000E49120FF03C0E295EF703F5FEF708E2F8C
:101D700090E0EA3010F0C79601C0C0968D939D9315
:101D80002F5F243149F74FBF8091E800877F809310
:101D9000E8006AE270E0CE0101960E94170D16C0BD
:101DA0006091530470915404AE014F5F5F4F0E94E5
:101DB000D70BBC01892B09F441C09091E800977FB3
:101DC0009093E80089819A810E94750D8091E800C6
:101DD0008B778093E80032C0803881F58091E800ED
:101DE000877F8093E80080914A048093F10080917E
:101DF000E8008E7772CF811121C0809151049091BB
:101E0000520499270297D4F48091E800877F809349
:101E1000E8008091510480934A040E94780C8091DC
:101E20004A04811106C08091E30087FD02C081E071
:101E300001C084E080934E040E94FF098091E80075
:101E400083FF0AC08091E800877F8093E80080913B
:101E5000EB0080628093EB00AA960FB6F894DEBF89
:101E60000FBECDBFDF91CF911F9108950E94A40FA7
:101E70000E94AC0FE0EEF0E0808181608083E8EDAD
:101E8000F0E080818F77808319BCA7EDB0E08C9162
:101E90008E7F8C9380818F7E808310924D04089575
:101EA0000F931F93CF93DF930E94A40F0E94AC0F58
:101EB000C8EDD0E088818F778883888180688883A7
:101EC00088818F7D888319BC10924E0410924A0439
:101ED00010924C0410924B0400EE10E0F801808147
:101EE0008B7F808388818160888342E060E080E02E
:101EF0000E94430CE1EEF0E080818E7F8083E2EE71
:101F0000F0E0808181608083808188608083F80137
:101F100080818E7F8083888180618883DF91CF91EB
:101F20001F910F910895E8EDF0E080818F7E80830E
:101F3000E7EDF0E080818160808384E082BF81E012
:101F400080934D040C94500FE8EDF0E080818E7F7B
:101F500080831092E20008951092DA001092E1005E
:101F600008951F920F920FB60F9211242F933F9353
:101F70004F935F936F937F938F939F93AF93BF9391
:101F8000EF93FF938091E10082FF0BC08091E2000C
:101F900082FF07C08091E1008B7F8093E1000E9467
:101FA0007E108091DA0080FF1FC08091D80080FFF2
:101FB0001BC08091DA008E7F8093DA008091D90077
:101FC00080FF0DC080E189BD82E189BD09B400FEBA
:101FD000FDCF81E080934E040E94F20905C019BC38
:101FE00010924E040E94FB098091E10080FF19C00D
:101FF0008091E20080FF15C08091E2008E7F809387
:10200000E2008091E20080618093E2008091D8003C
:1020100080628093D80019BC85E080934E040E94B2
:10202000F60A8091E10084FF30C08091E20084FFD5
:102030002CC080E189BD82E189BD09B400FEFDCFDD
:102040008091D8008F7D8093D8008091E1008F7EB1
:102050008093E1008091E2008F7E8093E200809186
:10206000E20081608093E20080914A04882311F0AD
:1020700084E007C08091E30087FD02C081E001C0D9
:1020800083E080934E040E940B0B8091E10083FF5C
:1020900024C08091E20083FF20C08091E100877F0F
:1020A0008093E10082E080934E0410924A04809174
:1020B000E1008E7F8093E1008091E2008E7F80932B
:1020C000E2008091E20080618093E20042E060E003
:1020D00080E00E94430C0E94FE09FF91EF91BF91A6
:1020E000AF919F918F917F916F915F914F913F91B0
:1020F0002F910F900FBE0F901F9018950895CF93BA
:1021000080914E048823A1F0C091E900CF70909196
:10211000EC00892F817090FD80E8C82B1092E900B7
:102120008091E80083FD0E94D60DCF70C093E90036
:10213000CF91089590935C0380935B030895E091A1
:102140005B03F0915C03309721F00190F081E02D6A
:10215000099480E00895EF92FF920F931F93CF931D
:10216000DF93E0915B03F0915C033097B1F18C0158
:102170000280F381E02D09958091390482FF2DC002
:1021800080FF04C089ED93E00E946405E80118E037
:1021900083EDE82E83E0F82E8091390480FF0BC098
:1021A00088811F928F93FF92EF920E94FD050F90FE
:1021B0000F900F900F90115021961111EDCF80913B
:1021C000390480FF0AC081ED93E0DF91CF911F9128
:1021D0000F91FF90EF900C946405DF91CF911F91C8
:1021E0000F91FF90EF900895E0915B03F0915C03F5
:1021F000309721F00480F581E02D09940895CF9364
:10220000DF932091590330915A032817390709F1B8
:1022100090935A0380935903E0915B03F0915C0320
:102220003097B9F0EC010680F781E02D0995809197
:10223000390482FF0EC080FF0CC0DF93CF9383EC84
:1022400093E09F938F930E94FD050F900F900F9046
:102250000F90DF91CF910895CF93DF932091570393
:10226000309158032817390709F190935803809348
:102270005703E0915B03F0915C033097B9F0EC01F8
:102280000084F185E02D09958091390482FF0EC00C
:1022900080FF0CC0DF93CF9383EB93E09F938F93EA
:1022A0000E94FD050F900F900F900F90DF91CF913E
:1022B00008950C9405120E943A1E0C945206BF9287
:1022C000CF92DF92EF92FF920F931F93CF93DF9302
:1022D00000D000D01F92CDB7DEB70E94DA060EE51F
:1022E00013E0F12C8F2D0E948507B82EF801C080D5
:1022F000C82639F4F3940F5F1F4FF0E1FF12F2CFBD
:1023000030C08091390481FD0E941A12D12CEE2434
:10231000E3948C2D8E21F9F0D982FA8291E08B2DF5
:102320008E2109F490E09B830E94431E8160782FE8
:102330009D838C8349815A816B818D810E945012CB
:1023400049815A816B817C818D810E94BB1DF8017E
:1023500080818E258083D394EE0CF8E0DF12D9CFF4
:10236000C9CF8FEF89838A831B820E94431E8160BD
:10237000782F9D838C8349815A816B818D810E9446
:1023800050120E94BA1D0E94E7200E949F10909157
:102390005D03891741F10E949F1080935D03909126
:1023A000390492FF0EC090FF0CC01F928F9384EEF1
:1023B00093E09F938F930E94FD050F900F900F90D5
:1023C0000F9080915D030F900F900F900F900F90E2
:1023D000DF91CF911F910F91FF90EF90DF90CF9001
:1023E000BF900C94CC1D0F900F900F900F900F90FA
:1023F000DF91CF911F910F91FF90EF90DF90CF90E1
:10240000BF9008950C948B0708950895CF93C62F1D
:102410000E94850721E030E002C0220F331FCA95D9
:10242000E2F790E02823392381E0232B09F480E0B0
:10243000CF910895EF92FF920F931F93CF93DF9365
:102440008AEF93E00E946405C0E0D0E089E2E82EC4
:1024500081E0F82E0FEE13E08C2F0E9485070E947A
:10246000A71DFF92EF921F928F93DF93CF931F933D
:102470000F930E94FD0521968DB79EB708960FB663
:10248000F8949EBF0FBE8DBFC031D10529F7DF91F3
:10249000CF911F910F91FF90EF90089508950895A7
:1024A000CF93DF93CDB7DEB72B970FB6F894DEBF8F
:1024B0000FBECDBF942F4F83252F588769877A870A
:1024C0008B874A855B85452B31F02F3F31F481E0C6
:1024D0009F3F19F403C081E001C080E080FD07C088
:1024E0004F81588569857A858B850E94BB1DDE01E9
:1024F000119686E0FD0111928A95E9F785E0FE01CB
:10250000379601900D928A95E1F749815A816B8146
:102510007C818D819E810E941C1A2B960FB6F894A7
:10252000DEBF0FBECDBFDF91CF910895CF93DF9374
:10253000882309F4EEC0C82F8EE78C0F833018F57E
:10254000C23829F0C33831F0C4E0D7E405C0C2E096
:10255000D9E302C0C1E0D3E50E949F108C2309F0AB
:10256000D8C08D2F0E94041D0E947C1D2FEF81EE8C
:1025700094E0215080409040E1F700C000008D2F92
:102580000E94211D0CC08CEF8C0F813A60F48C2FBF
:102590000E9411248111BDC08C2F0E94041DDF9167
:1025A000CF910C947C1D80E28C0F883048F4C7706A
:1025B00081E001C0880FCA95EAF70E94421DEFCF63
:1025C0008BE58C0F833080F4C53A29F0C63A31F0A0
:1025D00083E890E005C081E890E002C082E890E0E6
:1025E000DF91CF910C94FF1088E58C0F873108F0B4
:1025F00090C0C83A09F445C0C93A09F445C0CA3A7E
:1026000009F445C0CB3A09F445C0CC3A09F445C0B9
:10261000CD3A09F445C0CE3A09F445C0CF3A09F4A1
:1026200045C0C13B09F445C0C03B09F445C0C23BAD
:1026300009F445C0C33B09F445C0C43B09F445C097
:10264000C53B09F445C0C63B09F445C0C73B09F486
:1026500045C0C83B09F445C0C93B09F445C0CA3B65
:1026600009F445C0CB3B09F445C0CC3B09F445C057
:10267000CD3B09F445C0CE3B09F445C080E090E075
:1026800044C082EE90E041C089EE90E03EC08AEE08
:1026900090E03BC085EB90E038C086EB90E035C021
:1026A00083EB90E032C084EB90E02FC087EB90E0AA
:1026B0002CC08CEC90E029C08DEC90E026C083E823
:1026C00091E023C08AE891E020C082E991E01DC03A
:1026D00084E991E01AC081E292E017C083E292E0BF
:1026E00014C084E292E011C085E292E00EC086E25E
:1026F00092E00BC087E292E008C08AE292E005C057
:102700008FE690E002C080E790E0DF91CF910C94DB
:102710002C11DF91CF910895CF93DF93882309F493
:102720004FC09EE7980F933000F5823829F0833828
:1027300031F0C4E0D7E405C0C2E0D9E302C0C1E093
:10274000D3E50E949F108C23D9F18D2F0E94041D88
:102750000E947C1D2FEF81EE94E02150804090403C
:10276000E1F700C000008D2F04C09CEF980F913A54
:1027700018F40E94211D0DC090E2980F983068F463
:10278000877091E001C0990F8A95EAF7892F0E941E
:10279000481DDF91CF910C947C1D9BE5980F9330E1
:1027A00030F480E090E0DF91CF910C94FF10885AD4
:1027B000873130F480E090E0DF91CF910C942C11C0
:1027C000DF91CF910895882321F00E94421D0C943F
:1027D0007C1D0895882321F00E94481D0C947C1DC7
:1027E00008950E94621D0E94311D0E947C1D0E945E
:1027F0008C210E945A2080E090E00E94FF1080E02F
:1028000090E00C942C110E94521D0C94F113CF9265
:10281000DF92EF92FF920F931F93CF93DF9300D03D
:1028200000D01F92CDB7DEB76C010E94CE1D811182
:1028300018C385E0F601DE01119601900D928A958C
:10284000E1F7F60140815181238134812115310561
:1028500031F05F3F31F481E04F3F19F403C081E074
:1028600001C080E080FDFDC2F601F280E580E294C7
:102870008FE0E82249835A83FB82722F3D832C83A9
:102880006F2D8D810E94801C8C010E947F1C0E94F4
:102890006F1BE12FE295EF708E2F90E0FC01E05A64
:1028A000FF4F0C94C026812F807F1F70882311F06A
:1028B0001295107FFF20B9F0112329F0812F0E947B
:1028C000551D0E947C1D802F0F900F900F900F9030
:1028D0000F90DF91CF911F910F91FF90EF90DF90BC
:1028E000CF900C949612802F0E948C13112309F420
:1028F000B8C2812F0E945B1D0F900F900F900F9018
:102900000F90DF91CF911F910F91FF90EF90DF908B
:10291000CF900C947C1D812F807F1F70803211F02E
:102920001295107F002319F0013009F12BC0FF2010
:10293000A9F0EE2059F1F1E0812FEF1228C00F909D
:102940000F900F900F900F90DF91CF911F910F91EB
:10295000FF90EF90DF90CF900C94651DEE2021F05A
:1029600021E0E21609F47DC20E94681D4DC0FF20DF
:10297000E9F085E08E1508F474C20E943F1D8123A2
:1029800029F042C0FF20F1F1E11015C0812F0F9016
:102990000F900F900F900F90DF91CF911F910F919B
:1029A000FF90EF90DF90CF900C94E31394E09E158E
:1029B00008F457C229C0F601858180FF13C08F70CB
:1029C0008583E4CF003F09F489C108F055C180E454
:1029D000800F803208F459C1FF2009F4EAC1EE20CB
:1029E00009F49AC1802F0E949612093309F0DAC1C6
:1029F000FFEF21EE84E0F15020408040E1F700C07D
:102A000000002FC2E110D7C1812F59C1812F8695B7
:102A10008695837019F08130B9F023C2FF2019F038
:102A2000C801937002C080E090E00F900F900F906B
:102A30000F900F90DF91CF911F910F91FF90EF902A
:102A4000DF90CF900C94FF10FF2019F0C801937015
:102A500002C080E090E00F900F900F900F900F90C9
:102A6000DF91CF911F910F91FF90EF90DF90CF906A
:102A70000C942C11802FFF2019F00E946D1F02C0B2
:102A80000E94D51F0F900F900F900F900F90DF9125
:102A9000CF911F910F91FF90EF90DF90CF900C940A
:102AA0005A20812F837009F070C0F110DAC1202FF5
:102AB000229526952770220F220F602F6F70862F88
:102AC00090E0A0E0B0E06C017D01022E04C0CC0CCF
:102AD000DD1CEE1CFF1C0A94D2F704FF12C08FE02D
:102AE00090E0A0E0B0E004C0880F991FAA1FBB1FB0
:102AF0002A95D2F7BC01CD0160957095809590958F
:102B000003C060E070E0CB0116951695137012308B
:102B1000B1F040F56C297D298E299F29113031F1C2
:102B20000F900F900F900F900F90DF91CF911F910A
:102B30000F91FF90EF90DF90CF900C94941B6C2935
:102B40007D298E299F290F900F900F900F900F9045
:102B5000DF91CF911F910F91FF90EF90DF90CF9079
:102B60000C94AE1B0E94941BC701B6010F900F90EE
:102B70000F900F900F90DF91CF911F910F91FF90C9
:102B8000EF90DF90CF900C947A1BFF2019F0812FEB
:102B9000817001C08695882309F463C1202F229596
:102BA00026952770220F220F602F6F70862F90E0DE
:102BB000A0E0B0E06C017D01022E04C0CC0CDD1C55
:102BC000EE1CFF1C0A94D2F704FF12C08FE090E0C5
:102BD000A0E0B0E004C0880F991FAA1FBB1F2A9570
:102BE000D2F7BC01CD01609570958095909503C09A
:102BF00060E070E0CB011695169513701230B1F0BD
:102C000040F56C297D298E299F29113031F10F90D3
:102C10000F900F900F900F90DF91CF911F910F9118
:102C2000FF90EF90DF90CF900C945B1C6C297D2976
:102C30008E299F290F900F900F900F900F90DF918A
:102C4000CF911F910F91FF90EF90DF90CF900C9458
:102C50006D1C0E945B1CC701B6010F900F900F9076
:102C60000F900F90DF91CF911F910F91FF90EF90F8
:102C7000DF90CF900C94491C023F09F45EC008F429
:102C800049C0033F09F46CC0A7CE902F9071E92E84
:102C9000812F8F71FF2051F00E94E21B802FEE20C8
:102CA00019F08295807F73CE8F7071CE0E94031CC5
:102CB000802FEE2019F08295807F01C08F700F90D9
:102CC0000F900F900F900F90DF91CF911F910F9168
:102CD000FF90EF90DF90CF900C94EA13FF20A9F0C3
:102CE000E4E0EE1508F4BDC0812F8F710F900F90B6
:102CF0000F900F900F90DF91CF911F910F91FF9048
:102D0000EF90DF90CF900C94281CF5E0FE1508F4AE
:102D1000A8C0EACFFF2099F0812F8F710F900F90FC
:102D20000F900F900F90DF91CF911F910F91FF9017
:102D3000EF90DF90CF900C94E21BFF2069F3812F7E
:102D40008F710F900F900F900F900F90DF91CF9198
:102D50001F910F91FF90EF90DF90CF900C94031C88
:102D6000FF2089F0812F8F710F900F900F900F909F
:102D70000F90DF91CF911F910F91FF90EF90DF9017
:102D8000CF900C94CD1B0F900F900F900F900F9041
:102D9000DF91CF911F910F91FF90EF90DF90CF9037
:102DA0000C94C81B033509F423CE073409F059C02D
:102DB0001FCEEE2021F2802F0F900F900F900F90DA
:102DC0000F90DF91CF911F910F91FF90EF90DF90C7
:102DD000CF900C948C13412F4F70602FC6010E942E
:102DE000E71E0F900F900F900F900F90DF91CF91F3
:102DF0001F910F91FF90EF90DF90CF900C94CA1A23
:102E000001112FC0FF2069F10E9403142FEF80E70A
:102E100092E0215080409040E1F700C000000F9008
:102E20000F900F900F900F90DF91CF911F910F9106
:102E3000FF90EF90DF90CF900C94901E412F4F7039
:102E4000602FC6010F900F900F900F900F90DF91A1
:102E5000CF911F910F91FF90EF90DF90CF900C9446
:102E6000EA1E0F900F900F900F900F90DF91CF916F
:102E70001F910F91FF90EF90DF90CF9008951F93D7
:102E8000CF93DF9300D000D01F92CDB7DEB7942F41
:102E90004983252F5A836B837C838D834C815D818D
:102EA000452B31F02F3F31F481E09F3F19F403C0EF
:102EB00081E001C080E0182F117080FD24C049819D
:102EC0005A816B817C818D810E94801C292F2295E3
:102ED0002F702C3030F42A3048F42250223068F021
:102EE00013C02C3061F02F3051F00EC0803C28F020
:102EF000803E50F0815F833038F011E005C093FBD5
:102F0000112710F901C010E0812F0F900F900F9042
:102F10000F900F90DF91CF911F910895CF93DF9382
:102F200000D000D01F92CDB7DEB70F900F900F905A
:102F30000F900F90DF91CF910895CF93DF9300D042
:102F400000D000D0CDB7DEB726960FB6F894DEBF1E
:102F50000FBECDBFDF91CF9108951F93CF93DF9325
:102F6000C0916E0316E080916F03C81799F0D0E00E
:102F70001C9FF0011D9FF00D1124E059FC4F408172
:102F8000518162817381848195810E949D17219670
:102F9000C770E9CFDF91CF911F9108954091A003B1
:102FA0005091A1036091A2037091A3038091A403A7
:102FB0009091A5030C949D170F931F93CF93DF93CC
:102FC0008091A50382958F7009F05DC08091A20366
:102FD000882309F458C080916E0310916F036091AB
:102FE000A0037091A103C091A303D091A40391E029
:102FF0006F3F09F090E0292F06E0811709F443C0E4
:10300000209721F07F3F21F030E003C031E001C084
:10301000322F90E030FD34C0089FF001099FF00D81
:103020001124DF01A059BC4F11963C911197371321
:1030300027C03C91361324C012963C91129731114F
:103040001FC013964D915C9114974C1B5D0B483C2F
:103050005105B0F48091A5038F7080618093A50322
:10306000EB58FC4F80818F708061808380EA93E011
:103070000E940714DF91CF911F910F910C94AD170F
:1030800001968770BACFDF91CF911F910F9108956C
:103090009F92AF92BF92CF92DF92EF92FF920F93E7
:1030A0001F93CF93DF93CDB7DEB761970FB6F89438
:1030B000DEBF0FBECDBF8C0185E0F801DE011D969D
:1030C00001900D928A95E1F7F80140815181F280DB
:1030D000C380D4809091A0036091A1032091A303A9
:1030E0003091A4032115310531F06F3F31F481E0B7
:1030F0009F3F19F403C081E001C080E0F82FF17018
:103100009F2E80FD52C180EAA82E83E0B82EE09069
:10311000A203F601E21BF30BEE2009F4E8C0809154
:10312000A503E83CF10508F0A4C0282F207F09F092
:1031300053C0561313C0491311C0EF2CF1100EC029
:103140008F7080618093A5030E94CE17C5010E94F5
:1031500007148091A503F80185835BC1C114D104D4
:1031600031F05F3F31F481E04F3F19F403C081E05B
:1031700001C080E080FD03C081E08F2502C080E0B7
:1031800090E0F82FF170EF2E80FF1CC080916E034D
:1031900020916F0336E0821709F418C190E0389F40
:1031A000F001399FF00D1124E059FC4F6181561355
:1031B00006C06081461303C06281F61203C0019607
:1031C0008770E9CFEF2CFF2009F423C18091A5037C
:1031D00081608093A50362C0561306C0491304C0E2
:1031E000F11002C0F801A7C04D875E87FF867C2DD5
:1031F000D98AC88A6F2D89890E943F17882399F13F
:10320000FF2089F12091A503822F82958F7090E095
:10321000029774F08091A0039091A10398878F8307
:103220001986DB86CA862C87CE0107960E94071472
:1032300086E0F801A0EAB3E001900D928A95E1F7EB
:103240000E94DC170E94CE1711C0561749F14D8716
:103250005E87FF867C2DD98AC88A6F2D89890E9456
:103260003F1781112CC0C8010E940714EE24E3947B
:10327000D0C0282F207F49F77C2DD98AC88A6F2D8E
:1032800089890E948E1780EA93E00E94071486E0E5
:10329000F50111928A95E9F70E94CE17E12CB9C089
:1032A0004913D5CFF110D3CFF8018583C8010E940F
:1032B000071486E0F50111928A95E9F7AAC0FF206C
:1032C00091F22091A503822F82958F7090E0029752
:1032D0000CF4AECF8091A0039091A1039A838983CF
:1032E0001B82DD82CC822E83CE0101969FCFE83CEB
:1032F000F10508F04BC0EF2CFF2009F4B4CF5613B2
:1033000030C049132EC02091A50320FD21C0822F7B
:1033100082958F70482F50E041155105C9F0F80192
:1033200025834F30510541F08F5F982F9295907F04
:10333000822F8F70892B8583C8010E94071486E035
:10334000F801A0EAB3E001900D928A95E1F72AC056
:1033500086E0F801A0EAB3E001900D928A95E1F7CA
:1033600058C04D875E87FF867C2DD98AC88A6F2D0D
:1033700089890E943F1781115BCF8091A5038160ED
:103380008093A503C8010E94071443C07C2DD98AED
:10339000C88A6F2D89890E948E1786E0F5011192E7
:1033A0008A95E9F70E94CE1734C0FF2009F45BCF5D
:1033B0004D875E87FF867C2DD98AC88A6F2D8989C3
:1033C0000E943F17882309F44ECF32CF7C2DD98A33
:1033D000C88A6F2D89890E94801C292F22952F7001
:1033E000223028F49F7039F0811105C00BC02430C1
:1033F00028F49F7049F4805E883020F0C8010E9454
:1034000007149E2CE92C05C0F8019581907F99F74F
:10341000F9CF8E2D61960FB6F894DEBF0FBECDBFEB
:10342000DF91CF911F910F91FF90EF90DF90CF90A0
:10343000BF90AF909F9008951F93CF93DF93CDB728
:10344000DEB72C970FB6F894DEBF0FBECDBF4F830B
:10345000588769877A878B879C87CE0107960E9459
:1034600048188823D1F09F8188852A853B85232BA6
:1034700031F08F3F31F481E09F3F19F403C081E0C8
:1034800001C080E080FD47C04F81588569857A85FD
:103490008B859C850E949D173EC086E0FE01379675
:1034A000DE01119601900D928A95E1F7FF81E88582
:1034B0006A857B856115710531F0EF3F31F481E05C
:1034C000FF3F19F403C081E001C080E080FD23C00C
:1034D00020916F0330E0C9010196877099274091D0
:1034E0006E0350E084179507F1F1F983EA837D8339
:1034F0006C8396E0929FD001939FB00D1124A05948
:10350000BC4FFE01319601900D929A95E1F78093A0
:103510006F030E94AD1716E080916E0390916F03C8
:10352000891771F1189FC001112480599C4F0E9486
:103530004818882329F1E0916E031E9FF0011124A1
:10354000E059FC4F40815181628173818481958172
:103550000E949D1780916E0390E0019687709927D5
:1035600080936E03D9CF0E94031410926F031092C0
:103570006E03E0EAF3E086E0DF011D928A95E9F749
:103580002C960FB6F894DEBF0FBECDBFDF91CF9162
:103590001F910895DF92EF92FF920F931F93CF93A5
:1035A000DF93FC01892B09F488C0E12CF12CDD2488
:1035B000D394EF0121968491853709F460C058F4C3
:1035C000843708F04EC0843008F068C08130D1F0F4
:1035D000823071F172C0883709F45BC050F48637CD
:1035E00009F453C0873709F068C08E2D0E944F1D23
:1035F00052C09CE7980F903708F05FC08F770E9409
:103600008C134EC08F010E5F1F4FFE01849190E21C
:10361000980F983050F48770FD2D01C0FF0F8A95E8
:10362000EAF78F2F0E94551D15C00E94961214C0F4
:103630008F010E5F1F4FFE01849190E2980F98302A
:1036400068F48770FD2D01C0FF0F8A95EAF78F2F70
:103650000E945B1D0E947C1DE80122C00E948C1309
:10366000FBCFCF010296FE01C491CC2361F0EFE9BC
:10367000FFE03197F1F700C00000C150F6CFCF0155
:103680000296FE01F490EC010BC00E943F1DE82E53
:1036900007C00E94521D0E947C1D02C00E9496120B
:1036A0008F2D882341F0EFE9FFE03197F1F700C05B
:1036B00000008150F6CFFE017CCFDF91CF911F91AA
:1036C0000F91FF90EF90DF90089560932604709320
:1036D000270480932804909329040C94CB1D08950B
:1036E00060932A0470932B0480932C0490932D04F0
:1036F0000C94CA1D0F931F9300912A0410912B0460
:1037000020912C0430912D04602B712B822B932B54
:1037100060932A0470932B0480932C0490932D04BF
:103720001F910F910C94CA1D0F931F9300912A04AF
:1037300010912B0420912C0430912D0460237123CF
:103740008223932360932A0470932B0480932C0488
:1037500090932D041F910F910C94CA1D0F931F93EA
:1037600000912A0410912B0420912C0430912D04F7
:10377000602771278227932760932A0470932B0474
:1037800080932C0490932D041F910F910C94CA1DCB
:1037900060E070E0CB010C94651B0F931F9341E038
:1037A00050E060E070E08A019B0104C0000F111F2F
:1037B000221F331F8A95D2F7C901B8011F910F91BB
:1037C0000C94651B0F931F9341E050E060E070E0A4
:1037D00004C0440F551F661F771F8A95D2F780914A
:1037E000260490912704A0912804B09129048A010D
:1037F0009B01082B192B2A2B3B2BC901B8011F91C8
:103800000F910C94651B0F931F9341E050E060E013
:1038100070E004C0440F551F661F771F8A95D2F7CA
:10382000409550956095709580912604909127045D
:10383000A0912804B09129048A019B01082319232F
:103840002A233B23C901B8011F910F910C94651BDA
:103850000F931F9341E050E060E070E004C0440F1C
:10386000551F661F771F8A95D2F780912604909185
:103870002704A0912804B09129048A019B010827FC
:1038800019272A273B27C901B8011F910F910C94D2
:10389000651B0F931F93009126041091270420911C
:1038A000280430912904602B712B822B932B1F91BC
:1038B0000F910C94651B0F931F9300912604109198
:1038C0002704209128043091290460237123822346
:1038D00093231F910F910C94651B0F931F930091DD
:1038E0002604109127042091280430912904602790
:1038F0007127822793271F910F910C94651B0895C0
:103900008F929F92AF92BF92DF92EF92FF920F93AE
:103910001F93CF93DF9300D000D01F92CDB7DEB7B7
:103920006B837C838D838A018C819D81892B31F00F
:103930001F3F31F481E04F3F19F403C081E001C023
:1039400080E080FF03C080E090E04DC08B81882341
:10395000D1F18090260490902704A0902804B09084
:10396000290480912A0490912B04A0912C04B091F9
:103970002D04882A992AAA2ABB2A8FE1E82EF12C45
:10398000D501C4010E2C04C0B695A79597958795CF
:103990000A94D2F780FD06C081E0E81AF10880F7AA
:1039A000D12C07C0DE2CB8018E2D0E94BF1E0197BE
:1039B00099F388E0189FF0011124EA55FC4FE00FBD
:1039C000F11DD08209C088E0189FF0011124EA554A
:1039D000FC4FE00FF11DD08009831A8369817A8141
:1039E0008D2D0E94BF1E0F900F900F900F900F9083
:1039F000DF91CF911F910F91FF90EF90DF90BF90DB
:103A0000AF909F908F9008952091120130911301F3
:103A1000F90132969FEF40E05191851789F09F3F61
:103A200019F4511101C0942F4F5F4630A9F79F3F01
:103A300039F0F901E90FF11D97FDFA958283089598
:103A40000895E0911201F09113019F012A5F3F4F09
:103A50009281891301C012823196E217F307C1F7F0
:103A6000089581E090E0E0911201F0911301E80FD8
:103A7000F91F1082019688309105A9F70895809169
:103A80003804089590913804892B80933804089560
:103A90008095909138048923809338040895809309
:103AA0003804089510923804089590913704892BB2
:103AB00080933704089580959091370489238093EB
:103AC0003704089510923704089580932E040895C2
:103AD00010922E0408958091120190911301FC011F
:103AE00031969C01285F3F4F80E0919191118F5F4B
:103AF000E217F307D1F70895E0911201F091130155
:103B0000809138048083E0911201F091130190813B
:103B100080913704892B808380912E04882361F063
:103B2000E0911201F09113019081892B80830E9412
:103B30006B1D811110922E0480911201909113013E
:103B40000C94AB10909335018093340108958295C5
:103B5000982F937344E0949F900111248C7C869558
:103B60008695282B822F8575880F2A7A2695822B99
:103B7000089508950895CF93DF9300D000D01F9249
:103B8000CDB7DEB70F900F900F900F900F90DF9191
:103B9000CF910895089508950C94021280E008953D
:103BA00080914E04843021F110923A0420E488E19F
:103BB00090E00FB6F894A895809360000FBE209314
:103BC000600083B7817F846083BF83B7816083BFD8
:103BD0007894889583B78E7F83BF0FB6F894A895A5
:103BE00080916000886180936000109260000FBE39
:103BF0000895CF930E944E120E94DA060E944F123F
:103C0000C0E08C2F0E948507811104C0CF5FC031B6
:103C1000C1F701C081E0CF9108950E9404120C9475
:103C200003141F920F920FB60F9211248F939F933C
:103C3000AF93BF9380913A04811113C080913B04EC
:103C400090913C04A0913D04B0913E044196A11D89
:103C5000B11D80933B0490933C04A0933D04B0932A
:103C60003E04BF91AF919F918F910F900FBE0F9027
:103C70001F90189582E084BD93E095BD9AEF97BDA3
:103C800080936E0008952FB7F89480913B04909133
:103C90003C04A0913D04B0913E042FBF08952FB77E
:103CA000F89460913B0470913C0480913D049091A4
:103CB0003E042FBF08959C014FB7F89480913B04B8
:103CC00090913C04A0913D04B0913E044FBF821BF3
:103CD000930B089578941F920F920FB60F921124B0
:103CE0008F939F93AF93BF9380913B0490913C043B
:103CF000A0913D04B0913E040196A11DB11D809399
:103D00003B0490933C04A0933D04B0933E04BF91C8
:103D1000AF919F918F910F900FBE0F901F901895AC
:103D20000E94360FF89487E797E7909301088093F5
:103D3000000887E090EBDC018093570490935804CF
:103D4000A0935904B0935A049CE088E10FB6F8940C
:103D5000A895809360000FBE90936000FFCFE82F7E
:103D6000F0E088E0989FE00DF11D1124E052FF4F34
:103D70008491982F92959F708F7097700895CF932C
:103D8000C82FCB010E94AF1E40E1949F90011124E7
:103D9000282B203831051CF080E090E016C0977089
:103DA000E92FF0E098E0C99FE00DF11D112494E0A7
:103DB000EE0FFF1F9A95E1F78F70E80FF11DEE0FE0
:103DC000FF1FE050F84985919491CF91089580E0CC
:103DD00090E0089508958091410480FF0BC06091A8
:103DE000170185E0689FB001112475956795759559
:103DF00067952BC081FF09C06091170185E0689F1E
:103E0000B00111247595679520C082FF07C06091AD
:103E1000170185E0689FB001112417C090914204FA
:103E20009923D1F060911601961788F72091170118
:103E300085E0289F90011124929FA001939F500D2F
:103E4000112470E0CA010E94AC266038710540F46C
:103E50006115710519F406C065E070E0862F0895BC
:103E60008FE7089581E008958091410480FF08C0A4
:103E70006091150170E0759567957595679521C0FE
:103E800081FF06C06091150170E07595679519C0B6
:103E900082FF04C06091150170E010C0909142044F
:103EA000992399F0609114019617A0F7809115015C
:103EB000899FC001112470E00E94AC266038710512
:103EC00040F46115710519F406C061E070E0862FB9
:103ED00008958FE7089581E00895803F21F40E94BE
:103EE000EB1E819504C0813F29F40E94EB1E809354
:103EF00045040895823F21F40E94EB1E819504C081
:103F0000833F29F40E94EB1E809344040895893F67
:103F100019F40E94341F05C08A3F31F40E94341FF7
:103F200081958093460408958B3F21F40E94341FAD
:103F3000819504C08C3F29F40E94341F809347046C
:103F40000895843F21F480914304816017C0853F28
:103F500021F480914304826011C0863F21F4809156
:103F6000430484600BC0873F21F480914304886040
:103F700005C0883F31F480914304806180934304FD
:103F800008958D3F21F48091410481600BC08E3FE4
:103F900021F480914104826005C08F3F29F4809113
:103FA00041048460809341040895803F39F48091F6
:103FB000450487FF6CC01092450469C0813F29F415
:103FC000809145041816BCF362C090914404823F6E
:103FD00029F497FF5CC01092440459C0833F19F440
:103FE0001916CCF354C0893F41F480914604181649
:103FF0000CF04DC0109246044AC08A3F29F48091CB
:10400000460487FF44C0F6CF8B3F39F480914704C4
:1040100087FF3DC0109247043AC08C3F29F480913D
:1040200047041816BCF333C0843F21F48091430445
:104030008E7F17C0853F21F4809143048D7F11C08E
:10404000863F21F4809143048B7F0BC0873F21F48E
:1040500080914304877F05C0883F31F480914304F9
:104060008F7E8093430413C08D3F21F480914104DF
:104070008E7F0BC08E3F21F4809141048D7F05C05F
:104080008F3F29F4809141048B7F8093410480917C
:10409000440481110EC08091450481110AC08091B1
:1040A0004604811106C080914704811102C010921C
:1040B000420408958091390483FF7EC08EE294E02B
:1040C0000E946405809143041F928F9389E294E0DB
:1040D0009F938F930E94FD0587E294E00E94640500
:1040E00080914404282F082E000C330B3F938F93AC
:1040F00084E294E09F938F930E94FD0582E294E016
:104100000E94640580914504282F082E000C330B73
:104110003F938F938FE194E09F938F930E94FD05CF
:104120008DE194E00E94640580914604282F082EBA
:10413000000C330B3F938F938AE194E09F938F930E
:104140000E94FD0588E194E00E9464058091470487
:10415000282F082E000C330B3F938F9385E194E0BA
:104160009F938F930E94FD0582E194E00E94640575
:10417000809142041F928F938FE094E09F938F93DE
:104180000E94FD058DE094E00E9464058091410449
:104190001F928F938AE094E09F938F930E94FD0576
:1041A00087E094E00E9464058DB79EB74C960FB6E9
:1041B000F8949EBF0FBE8DBF83E494E00E94F4107C
:1041C0000E94431E9093400480933F0408951F93E0
:1041D000CF93DF9380913F04909140040E945B1E37
:1041E000AC0190914204992321F02091180130E014
:1041F00006C0209119018AE0289F900111244217DE
:10420000530708F485C080914404C0914504D091BF
:10421000460410914704811107C0C11175C0D11126
:1042200073C0111171C074C09F3F19F09F5F9093CC
:104230004204181624F40E94EB1E809344048091DB
:10424000440487FF05C00E94EB1E819580934404BF
:104250001C1624F40E94EB1E8093450480914504B3
:1042600087FF05C00E94EB1E8195809345046091F5
:104270004404662331F1C0914504CC2311F1062E8C
:10428000000C770B880B990B0E94B32523E333E3D3
:1042900043E35FE30E9417260E947B25609344045A
:1042A0006C2FCC0F770B880B990B0E94B32523E35F
:1042B00033E343E35FE30E9417260E947B2560936C
:1042C00045041D1624F40E94341F809346048091F7
:1042D000460487FF05C00E94341F819580934604E1
:1042E000111624F40E94341F8093470480914704E0
:1042F00087FF05C00E94341F819580934704DF919A
:10430000CF911F910C945A209F3F09F08FCFA0CFDF
:10431000DF91CF911F910895E3E4F4E085E0DF01A0
:104320001D928A95E9F71092420410924104089573
:1043300081E596E00E9464051F9281E08F931F92B1
:1043400085E08F9383E096E09F938F930E94FD0515
:104350000F900F900F900F900F900F900895833053
:10436000E9F128F4813061F0823009F10895853057
:1043700009F462C008F449C0863009F474C0089595
:1043800080911901262F30E0280F311D2F3F310574
:1043900024F4680F6093190103C08FEF8093190113
:1043A000809119011F928F938CE395E072C08091E8
:1043B0001801262F30E0280F311D2F3F310524F43E
:1043C000680F6093180103C08FEF809318018091EC
:1043D00018011F928F938AE295E05BC080911701CC
:1043E000262F30E0280F311D2F3F310524F4680FB0
:1043F0006093170103C08FEF80931701809117011D
:104400001F928F9387E195E044C080911601262F7B
:1044100030E0280F311D2F3F310524F4680F6093E1
:10442000160103C08FEF80931601809116011F9231
:104430008F9382E095E02DC080911501262F30E00A
:10444000280F311D2F3F310524F4680F60931501AB
:1044500003C08FEF80931501809115011F928F93F8
:1044600089EE94E016C080911401262F30E0280FC9
:10447000311D2F3F310524F4680F6093140103C0F0
:104480008FEF80931401809114011F928F938EEC13
:1044900094E09F938F930E94FD050F900F900F90D3
:1044A0000F900895833081F128F4813059F08230E3
:1044B000D1F00895853009F449C0B8F1863009F487
:1044C00056C0089580911901681720F4861B8093C7
:1044D000190102C010921901809119011F928F9346
:1044E0008FEB94E054C080911801681720F4861B6C
:1044F0008093180102C010921801809118011F9238
:104500008F938DEA94E043C080911701681720F4DF
:10451000861B8093170102C010921701809117012A
:104520001F928F938AE994E032C080911601681738
:1045300020F4861B8093160102C010921601809110
:1045400016011F928F9385E894E021C08091150198
:10455000681720F4861B8093150102C01092150184
:10456000809115011F928F938CE694E010C080918A
:104570001401681720F4861B8093140102C0109266
:104580001401809114011F928F9381E594E09F9311
:104590008F930E94FD050F900F900F900F9008953C
:1045A000CF93C82F1F928F9386E597E09F938F93A9
:1045B0000E94FD0581E090E0A0E0B0E0BC01CD01EB
:1045C00004C0660F771F881F991FCA95D2F70E94F3
:1045D000701B0F900F900F900F90CF910C940314BD
:1045E000CF93873288F58E3108F00BC18E3009F4F5
:1045F00087C0D8F4873009F460C08B3009F44FC00D
:10460000863009F002C180913904817F8E7F8093CA
:1046100039048BE597E00E94640588E19AE00E94E6
:10462000640581E08093490446C0863109F4B0C036
:1046300020F4803109F47AC0E8C0893109F491C0CE
:104640008B3109F449C0E1C0883349F150F4893213
:1046500009F4D5C0853309F4D2C0873209F0D5C03A
:10466000CEC0833409F4CBC028F48A3308F4CDC01B
:104670008953C8C0883409F0C8C00E94031487E079
:104680009AE00E9464052FEF83ED90E32150804073
:104690009040E1F700C000000E94901E0CC082E82C
:1046A00097E041C08EEE99E00E9464058091390444
:1046B000816080933904C1E0ADC080913904C82F76
:1046C000C17080FFEFCF8AEF99E00E94640580916E
:1046D0003904817F8E7F3FC09091390491FBCC27B4
:1046E000C0F981E0C827892FC0FB81F98093390484
:1046F000CC2319F081EE99E029C083ED99E013C035
:104700009091390492FBCC27C0F981E0C827892F0A
:10471000C0FB82F980933904CC2319F084EC99E032
:1047200015C084EB99E00E946405C5CF90913904CF
:1047300093FBCC27C0F981E0C827892FC0FB83F900
:1047400080933904CC2351F088EA99E00E946405F3
:10475000809139048160809339045CC08BE999E0D1
:10476000E2CF8CE899E00E9464058CE599E00E9414
:10477000640586E199E00E94640580EF98E00E945C
:1047800064058BEA98E00E94640580E898E0CBCF4E
:1047900082E798E00E9464050E949F101F928F9309
:1047A00088E598E09F938F930E94FD058091110109
:1047B0001F928F9381E498E09F938F930E94FD0551
:1047C000809156031F928F938EE298E09F938F9370
:1047D0000E94FD050E944F1E9F938F937F936F93BE
:1047E00087E198E09F938F930E94FD058DB79EB758
:1047F00042960FB6F8949EBF0FBE8DBF5CCF80E08F
:1048000001C08D510E94D02256CF85E198E00E94D0
:104810006405C0E08C2FCF91089580E008950C943A
:104820000D240F931F93CF93C82F8091490481309B
:10483000B1F020F0823009F45BC052C160E070E05A
:104840008CE090E00E940612892BC9F4E0911201DD
:10485000F09113018081843409F044C110C060E0FC
:1048600070E08CE090E00E9406128C01892B39F4F4
:10487000E0911201F09113018081843461F48C2F56
:104880000E940F24811104C08C2F0E94F0222EC0A0
:1048900081E090E02BC08C2F0E940D24811124C157
:1048A000C431E1F070F4CB3081F0C031D1F40E941A
:1048B00098218EE497E00E94640582E08093490489
:1048C00013C1C93259F0C83361F48BE597E00E94F7
:1048D000640582E597E00E94640506C110924904D0
:1048E00004C08CE497E00E946405802F8170FFC0B3
:1048F000C43228F5CE3108F0C1C0CB30A1F1D0F4DC
:10490000C73009F0D3C08EE18093190182E3809310
:1049100018018AE08093170184E18093160188E0F2
:104920008093150188E28093140182EF95E00E9444
:104930006405BFC0C33149F1C431C1F0B7C0CB3445
:1049400009F4A9C028F4C93289F0C83361F0AEC0B7
:10495000C13509F49EC0C23509F499C0CE3409F0BE
:10496000A5C06AE09EC00E949821A3C0809148041F
:10497000882319F0109248049CC08FEF95E00E94A4
:10498000640581E080934904B2C089ED95E00E94FE
:10499000640587EC95E00E946405809119011F92DF
:1049A0008F9384EC95E09F938F930E94FD0582EC9A
:1049B00095E00E94640580EB95E00E94640580917B
:1049C00018011F928F938DEA95E09F938F930E9419
:1049D000FD058BEA95E00E9464058CE995E00E9454
:1049E0006405809117011F928F9389E995E09F9349
:1049F0008F930E94FD0587E995E00E94640586E893
:104A000095E00E946405809116011F928F9383E8C0
:104A100095E09F938F930E94FD0581E895E00E94A9
:104A200064058CE695E00E946405809115011F9253
:104A30008F9389E695E09F938F930E94FD0587E60B
:104A400095E00E94640580E595E00E9464058091F0
:104A500014011F928F938DE495E09F938F930E9492
:104A6000FD058BE495E00E9464058DB79EB74896DE
:104A70000FB6F8949EBF0FBE8DBF1BC0CE51EC2F5A
:104A8000F0E0E65DFE4F80818093480412C061E053
:104A900003C061E006C06AE0809148040E94AF2133
:104AA00008C0809148040E94522203C080EF95E024
:104AB00013C080914804882369F01F928F938AEE77
:104AC00095E09F938F930E94FD050F900F900F909C
:104AD0000F9004C087EE95E00E94640581E007C056
:104AE0001092490480E003C001E010E0FECECF91B7
:104AF0001F910F9108950E9482256894B1110C9422
:104B0000112608950E94F62588F09F5798F0B92F36
:104B10009927B751B0F0E1F0660F771F881F991FF2
:104B20001AF0BA95C9F714C0B13091F00E9410265E
:104B3000B1E008950C941026672F782F8827B85F6E
:104B400039F0B93FCCF3869577956795B395D9F74A
:104B50003EF490958095709561957F4F8F4F9F4F54
:104B60000895E89409C097FB3EF490958095709560
:104B700061957F4F8F4F9F4F9923A9F0F92F96E9A9
:104B8000BB279395F695879577956795B795F1111E
:104B9000F8CFFAF4BB0F11F460FF1BC06F5F7F4FBB
:104BA0008F4F9F4F16C0882311F096E911C07723CD
:104BB00021F09EE8872F762F05C0662371F096E8D6
:104BC000862F70E060E02AF09A95660F771F881FA5
:104BD000DAF7880F9695879597F9089557FD9058BD
:104BE000440F551F59F05F3F71F04795880F97FBB1
:104BF000991F61F09F3F79F087950895121613066B
:104C00001406551FF2CF4695F1DF08C01616170699
:104C10001806991FF1CF86957105610508940895CE
:104C2000E894BB2766277727CB0197F908950E9460
:104C30002A260C949B260E948D2638F00E949426EA
:104C400020F0952311F00C9484260C948A261124CC
:104C50000C9411260E94EE2570F3959FC1F3950FD9
:104C600050E0551F629FF001729FBB27F00DB11DF0
:104C7000639FAA27F00DB11DAA1F649F6627B00D80
:104C8000A11D661F829F2227B00DA11D621F739F69
:104C9000B00DA11D621F839FA00D611D221F749F77
:104CA0003327A00D611D231F849F600D211D822FBE
:104CB000762F6A2F11249F5750409AF0F1F08823E5
:104CC0004AF0EE0FFF1FBB1F661F771F881F915012
:104CD0005040A9F79E3F510580F00C9484260C9417
:104CE00011265F3FE4F3983ED4F386957795679558
:104CF000B795F795E7959F5FC1F7FE2B880F911D3C
:104D00009695879597F9089597F99F6780E870E0E1
:104D100060E008959FEF80EC089500240A94161631
:104D2000170618060906089500240A941216130699
:104D3000140605060895092E0394000C11F4882327
:104D400052F0BB0F40F4BF2B11F460FF04C06F5F43
:104D50007F4F8F4F9F4F089597FB072E16F40094B7
:104D600007D077FD09D00E94C62607FC05D03EF487
:104D7000909581959F4F0895709561957F4F089507
:104D8000EE0FFF1F0590F491E02D0994AA1BBB1BA9
:104D900051E107C0AA1FBB1FA617B70710F0A61B3B
:104DA000B70B881F991F5A95A9F780959095BC015C
:084DB000CD010895F894FFCF36
:104DB800054D020000FF1708B9088A084E081A08AE
:104DC80001012F042808140A321E407F227303F4BD
:104DD80002D20277029002A902000102030405062A
:044DE80007080900AF
:1068000088000000000000000400050006000700EA
:10681000080009000A000B000C000D000E000F001C
:1068200010001100120013001400150016001700CC
:10683000180019001A001B001C001D001E001F007C
:10684000200021002200230024002500260027002C
:10685000280029002A002B002C002D002E002F00DC
:1068600030003100000033003400000036003700F3
:10687000380082003A003B003C003D003E003F00F3
:106880004000410042004300440045004600000033
:10689000000049004A004E004C004D004B004F00E4
:1068A000500051005200000054005500560057009F
:1068B000580059005A005B005C005D005E005F00FC
:1068C00060006100620063000000650085006700F1
:1068D000680069006A00000000000000000000007D
:1068E0000000000000000000890087008A008B0083
:1068F000E000E100E200E3000000E500E600E70060
:00000001FF
